S01400006F7064726163687420332E332E7372656307
S113000045C0000060C000005EC000005CC000008D
S11300105AC0000058C0000056C0000054C0000080
S113002052C0000069C000004EC000004CC0000077
S11300304AC0000048C0000046C0000044C00000A0
S113004042C0000040C000003EC000003CC00000B0
S11300503AC0000038C0000036C0000034C00000C0
S113006032C0000030C000002EC000002CC00000D0
S11300702AC0000028C0000026C0000024C00000E0
S113008022C0000020C000001EC0000011241FBEBA
S1130090CFEFD0E1DEBFCDBF11E0A0E0B1E0E0E9F9
S11300A0F1E000E00BBF02C007900D92A230B1074F
S11300B0D9F721E0A2E0B1E001C01D92A430B2075B
S11300C0E1F75BD063C09CCF20E030E008C0EFECE8
S11300D0F7E03197F1F700C000002F5F3F4F28177A
S11300E03907ACF308958BE983BD87B7806887BF70
S11300F078948BE085BD08951F920F920FB60F92EE
S113010011242F933F938F939F9380910201909199
S1130110030101969093030180930201209102014F
S11301203091030180910001909101012817390752
S1130130D8F095B381E0892785BB10920301109212
S1130140020180910001909101010F9739F489E136
S113015090E0909301018093000106C08FE090E04D
S113016090930101809300019F918F913F912F9172
S11301700F900FBE0F901F9018958FEF84BB81E0F6
S113018085BBB1DF8AE090E09FDFFCCFF894FFCF1E
S10501900F005A
S9030000FC
